:100000000C9453000C9470000C9470000C947000CD
:100010000C9470000C9470000C9470000C947000A0
:100020000C9470000C94BC000C9470000C94700044
:100030000C9470000C9470000C9470000C94700080
:100040000C9470000C9455030C9443020C94FA0128
:100050000C94EF010C9470000C9470000C947000E0
:100060000C9470000C9470002025303278002531FB
:1000700058202531780043253032643A20006374DB
:10008000726C5F616C6C6F632825642920696478E9
:100090003D25640A007E0E0E0E0E1B1B1C0E1B1B44
:1000A0007E0E0E0E0E0011241FBECFEFD4E0DEBF79
:1000B000CDBF11E0A0E0B1E0E2EBF8E202C00590B4
:1000C0000D92A431B107D9F713E0A4E1B1E001C06A
:1000D0001D92A53BB107E1F70E947C000C945814D7
:1000E0000C9400008091140190E008950E948E030A
:1000F0000E94BA10A89508950E94B0010E9435038D
:100100000E949D0F409A789401C0A8950E940C10FF
:100110008823D9F30E94EC0C0E94CB0140980E94E6
:10012000DD020E9497080E947600F9CF9091140199
:100130009817F9F09630E9F0953011F48630C9F44B
:10014000809314010E94690480911401853029F480
:1001500045E060E280E00E94CF0D8091140186307E
:1001600029F446E060E280E00E94CF0D81E090E05B
:10017000089580E090E008951F920F920FB60F92BD
:1001800011248F939F93AF93BF938091AD038823E6
:1001900029F08091AD0381508093AD0380911501CA
:1001A000882329F581E080931501789480911601C8
:1001B0008F5F809316018091160190E0837090709C
:1001C000892B99F48091A5039091A603A091A70390
:1001D000B091A8030196A11DB11D8093A503909332
:1001E000A603A093A703B093A80310921501BF9193
:1001F000AF919F918F910F900FBE0F901F90189508
:100200001092A5031092A6031092A7031092A803C0
:10021000E0E7F0E010821092B00082E08093B1003D
:100220008081816080830895EF92FF920F931F93E6
:100230002091A5033091A6034091A7035091A803F4
:100240007C0100E010E0E20EF31E041F151F02C047
:100250000E947600C801B7010E94ED0D8823C1F30A
:100260001F910F91FF90EF900895EF92FF920F93DF
:100270001F932091A5033091A6034091A7035091AD
:10028000A8037C0100E010E0E20EF31E041F151F1E
:1002900001C0A895C801B7010E94ED0D8823C9F3DC
:1002A0001F910F91FF90EF90089520E030E0D90169
:1002B0000E940814802DF901E95EFE4FE0818E173F
:1002C00021F0D9010E2E0E941514A8952F5F3F4FE3
:1002D0002032310561F7089587E191E0089520E02B
:1002E00030E090911701982311F021E030E0C9012E
:1002F000089590911701982B909317010E94550132
:1003000008958095909117019823909317010E946A
:10031000550108958CEF9FE3FC0185919591A5917E
:10032000B491B070BC01CD010895EFEFFFE3E4910B
:100330008E2F90E00895F894FFCF90911C01943097
:1003400008F091E08FE0E7E1F1E011928A95E9F79A
:1003500088E180931B0190931C010E945501089530
:1003600080E2E7E1F1E0A0E0B0E0182E0E94101476
:100370008091190190911A018F5F9F4F11F40E9493
:100380009D01EAEFFFE39491892F81508E3F10F495
:1003900090936600089510923801809138018093FF
:1003A00037018091370180935A0180915A018093DF
:1003B0005901519A5098599A589A5A9882E08093C4
:1003C000C0001092C5008FE08093C40086E0809347
:1003D000C2008CEF8093C10080E090E008951F92EE
:1003E0000F920FB60F9211245A980F900FBE0F90D4
:1003F0001F9018951F920F920FB60F9211248F9392
:100400009F93EF93FF939091590180915A01981710
:1004100031F48091C1008F7D8093C1002BC05A9A26
:100420008091630187FF09C0809163018F7780937A
:1004300063018091C100816003C08091C1008E7F03
:100440008093C1008091C00080648093C000E091DF
:100450005A01F0E0E95CFE4F84A18093C6008091D0
:100460005A018F5F80935A0180915A01883010F0B1
:1004700010925A01FF91EF919F918F910F900FBEB3
:100480000F901F9018951F920F920FB60F92112484
:100490002F933F938F939F93EF93FF935A9B03C0A8
:1004A0008091C60030C0209137018091380130E042
:1004B00090E001972817390741F0809137018F317B
:1004C00079F480913801882359F4809138018F5F45
:1004D0008093380180913801803210F010923801F9
:1004E000E0913701F0E08091C600E95CFE4F828325
:1004F000809137018F5F809337018091370180327F
:1005000010F010923701FF91EF919F918F913F91E1
:100510002F910F900FBE0F901F901895482F06C077
:100520008091C10080628093C1007894A895209149
:10053000590180915A0130E090E00197281739075E
:1005400079F380915901873021F480915A018823F1
:1005500039F3E0915901F0E0E95CFE4F44A380914A
:1005600059018F5F8093590180915901883010F0B3
:10057000109259018091C10080628093C100842F44
:1005800090E0089590916301906890936301282F03
:100590002F77822F82958F70E0E0F1E0DF01A80FC6
:1005A000B11D822F8F70E80FF11D8C9190818927EA
:1005B000822B0E948E0290E00895909137018091E5
:1005C0003801981719F48FEF9FEF0895E0913801E3
:1005D000F0E0E95CFE4F9281F894809138018F5FE2
:1005E0008093380180913801803210F010923801E8
:1005F000892F90E0789408958BB190E09695879537
:1006000096958795817090700895EF92FF920F9361
:100610001F93BC01181619061CF58091A503909133
:10062000A603A091A703B091A8037B010027F7FCC4
:100630000095102FE80EF91E0A1F1B1F8091C100A4
:1006400088708093C1005A9A599A02C00E9476001D
:10065000C801B7010E94ED0D8823C1F30E94CB01B0
:100660001F910F91FF90EF9008951092C1001CBC54
:1006700083E084B915B881E087B992E098B98EEF2C
:100680008AB99BB90E940001A895E0E6F0E088E1F4
:1006900080838CE08083089584B1837C84B985B1A4
:1006A000837C85B984EE8CBD08951F920F920FB69E
:1006B0000F9211242F933F934F935F936F937F93E8
:1006C0008F939F93AF93BF93EF93FF93809110010C
:1006D000909111012FEF8F3F920749F0249A8EBD20
:1006E0000DB406FE07C024980E94150F03C024987D
:1006F0008FEF8EBD8EB50E94340EFF91EF91BF91AA
:10070000AF919F918F917F916F915F914F913F91A9
:100710002F910F900FBE0F901F901895809112018E
:100720008F3FB9F06091A9037091AA038091AB0348
:100730009091AC036C507E4F8F4F9F4F0E94ED0DF8
:10074000882339F0409A8FEF8093120180E090E087
:10075000089581E090E0089540E050E060E080E09E
:1007600090E00E94FF10409808950F931F93CF933D
:10077000DF938C018091A5039091A603A091A7031C
:10078000B091A8038093A9039093AA03A093AB030D
:10079000B093AC030E94CB0CDC01E8012A818B8171
:1007A000C82FD0E0D695DC2FCC27D795C795822FC0
:1007B00090E0C82BD92BF8018181853081F08630FB
:1007C00018F48330F9F405C0893079F08032D1F41F
:1007D00017C0822F0E94960015C00E948607CE0186
:1007E0000E94D00C0097C9F70DC0109759F0FD0179
:1007F000D283C18314821382E8018C81858302C075
:100800000E949B018091AE03882381F0F801208132
:1008100030E02F7730708091120190E0281739076F
:1008200029F48091AE0381508093AE03DF91CF9184
:100830001F910F910895FC018181893159F0209118
:10084000E8013091E9012115310551F0CF01F9019D
:100850000995089584818093EF0181E08093EE01F2
:100860000895CF93DF93E9012091E60192E1299F5A
:10087000F0011124E658FE4F682B608342834F70CD
:10088000DF01139603C089918D9341504423D9F71A
:1008900083E081838091E6018F5F8093E601809100
:1008A000E601863010F01092E6019091E601809109
:1008B000E701981759F48091E7018F5F8093E70172
:1008C0008091E701863010F01092E701DF91CF911F
:1008D0000895CF93DF93CDB7DEB72F970FB6F89477
:1008E000DEBF0FBECDBF0E947200833051F0843056
:1008F00051F09E012F5F3F4F823059F4198241E839
:100900000AC081E001C082E089839E012F5F3F4FD2
:1009100001C0198241E660E080E60E9431042F9612
:100920000FB6F894DEBF0FBECDBFDF91CF91089513
:10093000EF92FF920F931F93CF93DF93EC01E62E7C
:100940008A012115310519F48FEF9FEF43C0C901CA
:100950000E94C10F9093E9018093E801D093EB01CD
:10096000C093EA011092EE018EEF9FEF9093ED019C
:100970008093EC01FF24EE2029F0A8016E2D80E089
:100980000E94B90D84E08093AE0302C00E947600FD
:100990008091EE01882321F48091AE038823B1F782
:1009A0000E94B50F8111FF248091EE01882321F46C
:1009B000F39487E08F15F8F68091E8019091E901B2
:1009C0000E94C10F1092E9011092E8018091EC01A0
:1009D0009091ED01DF91CF911F910F91FF90EF90DA
:1009E0000895CF92DF92EF92FF920F931F93CF93D0
:1009F000DF93CDB7DEB726970FB6F894DEBF0FBEF4
:100A0000CDBF6C017A0161157105C9F0452BB9F0B4
:100A10008E010F5F1F4F86E0F80111928A95E9F76A
:100A2000C8010E94AD0DB701CE0103960E94AD0D25
:100A30002FEC35E0A80162E0C6010E9498042696DA
:100A40000FB6F894DEBF0FBECDBFDF91CF911F91DF
:100A50000F91FF90EF90DF90CF900895EF92FF926B
:100A60000F931F93CF93DF93CDB7DEB726970FB6C3
:100A7000F894DEBF0FBECDBF8C017E010894E11C4F
:100A8000F11CC7010E94AD0DF801138622E936E082
:100A9000A7016EE0C8010E94980426960FB6F8944C
:100AA000DEBF0FBECDBFDF91CF911F910F91FF90A1
:100AB000EF900895EF92FF920F931F93CF93DF93E0
:100AC000CDB7DEB726970FB6F894DEBF0FBECDBF09
:100AD0008C01FC01618172817E010894E11CF11C92
:100AE000C7010E94AD0DF801478150856681609570
:100AF0006078C7010E94930DA70163E080E00E9427
:100B0000B90DF8014781508566816078C7010E9460
:100B1000930DA70163E080E00E94B90D26960FB601
:100B2000F894DEBF0FBECDBFDF91CF911F910F9123
:100B3000FF90EF900895EF92FF920F931F93CF9342
:100B4000DF93CDB7DEB726970FB6F894DEBF0FBEA2
:100B5000CDBF7C01FC01618172818E010F5F1F4F4F
:100B6000C8010E94AD0DF701478150856681C8011B
:100B70000E94930DA80163E080E00E94B90D88E017
:100B8000F701818726960FB6F894DEBF0FBECDBF62
:100B9000DF91CF911F910F91FF90EF900895EF9209
:100BA000FF920F931F93CF93DF93DC01E091EA0153
:100BB000F091EB01309721F481E08093EE019FC02A
:100BC000EC018B81482F50E05695542F44275795C0
:100BD00047958A8190E0482B592B6981673008F44A
:100BE0008EC0693080F0693009F089C0528341833A
:100BF000148213828C818583838584608387873008
:100C000009F089C074C005E0E02EF12CEA0EFB1E4D
:100C1000ED018D8190E0982F8827990F990F8D0114
:100C2000095F1F4F2E8130E02F77307073E0220F65
:100C3000331F7A95E1F7282B392B8F8190E080774D
:100C4000907074E0959587957A95E1F7282B392B6C
:100C50006830E9F4548343838781908537FF02C06D
:100C6000906401C09F7B908787832F70307044E031
:100C7000220F331F4A95E1F7878190858F70282BCB
:100C8000392B308727838385826083872DC05283E9
:100C9000418383819481892B81F08781908537FFFF
:100CA00002C0906801C09F77908787832F70307053
:100CB00087819085807F282B392B30872783E70118
:100CC000888190E080749070880F991FED012C81CD
:100CD000282B26839385892F81608387D8018C9167
:100CE00080FD02C09360938783858730A1F481E003
:100CF0008093EE011092ED011092EC010CC0E09196
:100D0000E801F091E901309719F0CD01099503C090
:100D1000CD010E94B503DF91CF911F910F91FF90FC
:100D2000EF900895EF92FF920F931F93CF93DF936D
:100D3000DC01E091EA01F091EB01309721F481E0D0
:100D40008093EE01A8C0EC018B81482F50E05695AE
:100D5000542F4427579547958A8190E0482B592B6B
:100D60006981693061F06A3020F4673008F493C01B
:100D700014C0862F8E50823008F08DC00EC0528372
:100D8000418314821382ED018C8185838385846085
:100D90008387873009F08BC076C005E0E02EF12C08
:100DA000EA0EFB1EED018D8190E0982F8827990FA8
:100DB000990F8D01095F1F4F2E8130E02F77307022
:100DC00073E0220F331F7A95E1F7282B392B8F819F
:100DD00090E08077907074E0959587957A95E1F72B
:100DE000282B392B6F3011F06830E9F4548343839A
:100DF0008781908537FF02C0906401C09F7B9087F8
:100E000087832F70307044E0220F331F4A95E1F73B
:100E1000878190858F70282B392B30872783838596
:100E2000826083872DC05283418383819481892B83
:100E300081F08781908537FF02C0906801C09F775D
:100E4000908787832F70307087819085807F282BD3
:100E5000392B30872783E701888190E08074907078
:100E6000880F991FED012C81282B26839385892FCC
:100E700081608387D8018C9180FD02C09360938745
:100E800083858730A1F481E08093EE011092ED011B
:100E90001092EC010CC0E091E801F091E90130976B
:100EA00019F0CD01099503C0CD010E94B503DF9172
:100EB000CF911F910F91FF90EF900895FF920F93A4
:100EC0001F93CF93DF93182F062FEA010E94FC0295
:100ED0008823E1F7812F0E94C202802F0E948E0298
:100EE000182F9FE0F92EF02200E005C089910E94A2
:100EF0008E0218270F5F0F15C9F7812F0E948E02EF
:100F0000DF91CF911F910F91FF9008950F931F9341
:100F1000CF93DF93CDB7DEB72F970FB6F894DEBF30
:100F20000FBECDBF8C01892BF1F080E48983F801DD
:100F300021813281832F992787FD9A95482F8A83B3
:100F40002436310514F0406C4A83F80181818B838B
:100F50008081AE014F5F5F4F63EE80660E945E0747
:100F600087E0F80182872F960FB6F894DEBF0FBE98
:100F7000CDBFDF91CF911F910F910895BF92CF9276
:100F8000DF92EF92FF920F931F93CF93DF93CDB732
:100F9000DEB726970FB6F894DEBF0FBECDBF7C013B
:100FA0006B01009709F45FC06115710509F45BC01E
:100FB000FC018181928121858617970719F42830D9
:100FC00049F44EC0283019F487E0F7018187F70112
:100FD000D282C182C6010E94D00CDC01009709F1C7
:100FE0008E159F05F1F0FC0181819281F7019283BA
:100FF0008183FD0183819481F70194838383FD01C3
:101000008581F7018583FD018681F7018683FD01D6
:1010100087819085F70190878783CD010E9486079D
:101020001CC056E0B52E8E010F5F1F4FF8018B2DAF
:1010300011928A95E9F7F7011386B601C8010E945B
:10104000AD0D2FEC35E0A80161E0C7010E949804C6
:1010500097FF03C0F701B28606C088E0F7018287D8
:1010600081E090E002C080E090E026960FB6F89410
:10107000DEBF0FBECDBFDF91CF911F910F91FF90CB
:10108000EF90DF90CF90BF900895CF93DF93CDB7CF
:10109000DEB761970FB6F894DEBF0FBECDBF6F8984
:1010A000962F9F70AE01485E5F4F5A834983FA01C5
:1010B000292FDE01139604C080818D932150329632
:1010C0002223D1F7892F90E0880F991F480F591FCD
:1010D0005A834983AE014D5F5F4F8E890E945E0740
:1010E00061960FB6F894DEBF0FBECDBFDF91CF91F2
:1010F000089521E830E03F932F9391E69F93806617
:101100008F930E9445080F900F900F900F900895B5
:1011100022E830E03F932F9391E69F9380668F9370
:101120000E9445080F900F900F900F900895DF9246
:10113000EF92FF920F931F93CF93DF93CDB7DEB75C
:1011400026970FB6F894DEBF0FBECDBF9C018FEF80
:101150002F3F380799F090917801913108F0F1C351
:10116000E92FF0E0E959FE4F208380917901822731
:10117000809379019F5F90937801E3C30E94FC0202
:10118000882319F084E08093AD038091AD03882318
:1011900009F0DAC340917801242F30E08091670193
:1011A00090E08F70907002962817390709F004C3F9
:1011B00080917901882309F0FFC20E94CB0FD09063
:1011C00064018F3F21F48D2D0E9479080FC3409A4E
:1011D00061E08D2D0E94320D8C01009709F488C2C8
:1011E000FC018185863021F48D2D0E94790885C20D
:1011F000823018F482E0F801818790916701892F8D
:1012000082958F70853009F4DAC0863030F48230F0
:1012100071F0843009F06CC25DC0893009F411C2EC
:101220008E3009F4F9C0883009F062C2EFC0903204
:1012300019F4F801128661C280916801843209F1C3
:10124000853220F4813209F053C206C0803899F10A
:10125000813809F04DC235C0F0E6DF2A1F921F9297
:1012600080E390E09F938F9381E290E09F938F9330
:1012700083E68F93DF920E9445088DB79EB708964C
:1012800086C10E947200823011F481E009C0882377
:1012900011F482E005C0843011F488E001C080E0E0
:1012A00090E0E0E6DE2A9F938F9382E290E09F93A6
:1012B0008F9382E67CC00E947200882331F040E068
:1012C000A6C00E947200833019F40E94690415C2FE
:1012D00043E09DC080916801082F10E0000F111FAE
:1012E000000F111F8091690180FF02C00E5F1F4F28
:1012F00001FF03C080E1F82E01C0FF24B80187E69A
:1013000091E00E94AD0D2BE134E047E651E069E148
:1013100080E090E00E9498048091EF01823551F0C6
:1013200083351CF4873479F40AC0873651F082374C
:1013300051F402C090E8F92AE1E0FE2A04C0F0E886
:10134000FF2A22E0F22AB8016F5F7F4F87E691E023
:101350000E94AD0D2BE134E047E651E069E180E009
:1013600090E00E9498048091EF01823551F083351E
:101370001CF4873479F40AC0873651F0823751F46F
:1013800002C080E8F82A94E0F92A04C0E0E8FE2AC6
:10139000F8E0FF2A8F2D90E0169507951695079592
:1013A00020E6D22A9F938F931F930F9382E48F930B
:1013B000DF920E9445088DB79EB70696E8C06091FF
:1013C000680170E0A3E0660F771FAA95E1F700912E
:1013D000690110E0C80187709070682B792B81E05B
:1013E00090E0682779277E010894E11CF11CC70171
:1013F0000E94AD0D1B821C8203FF02C081E08C8322
:10140000A70166E080E00E94B90D77C142E060E28A
:1014100080E00E94CF0D71C18091690190E0F82EAB
:10142000EE2480916A0190E0E82AF92AEFEFFFE3C9
:10143000EE22FF2280916801833160F4813108F04F
:10144000C4C0873009F4A9C0803109F4E5C08823FD
:1014500089F04EC1803209F4FFC0813220F483311B
:1014600009F046C1DEC0813209F414C1823209F0AC
:101470003FC125C1F80181819281E816F90659F131
:101480008185883011F487E08187C7010E94D00CE4
:10149000DC01009701F180179107E9F0FC018181DF
:1014A0009281F80192838183FD0183819481F80107
:1014B00094838383FD018581F8018583FD01868105
:1014C000F8018683FD0187819085F80190878783E5
:1014D00087E0818704C0B701C8010E942E05F8018A
:1014E00085810E942A0E282F8B3148F08D3118F00B
:1014F0008E3729F402C062E003C064E001C060E0FE
:10150000F8018185883009F06860F801A681BA2F5A
:10151000BF772B51223078F4B111BD5F8B2F90E053
:1015200081709070E4E0880F991FEA95E1F7B69515
:10153000BF70B82B02C0B111BF5FF80187819085E1
:10154000292F221F2227221F2295207FAC0174E021
:10155000559547957A95E1F750E08F70282B30E04C
:10156000A078BA2B8B2F90E070E0F0E6DF2A5F9333
:101570004F933F932F939F938F937F936F9384EE1B
:101580008F93DF920E9445088DB79EB70A960FB6DB
:10159000F8949EBF0FBE8DBFB0C090E6D92A1F92AF
:1015A0001F921F921F9280E590E09F938F9383EE8E
:1015B0008F93DF920E944508EDB7FEB738960FB6BD
:1015C000F894FEBF0FBEEDBF98C0B701C8010E94DE
:1015D000BE07882309F491C040916B01842F90E0ED
:1015E0009C012071307054E0359527955A95E1F7AC
:1015F0008F709070880F991F282B822F8150823016
:1016000020F44078F80146831CC021112350407813
:10161000242BF801268368C080916B018F7880931A
:101620006B01B701C8010E94BE07882309F465C099
:1016300090916B01892F8F77813039F49078F80180
:101640009683C8010E945A0558C081118150907834
:10165000892BF801868348C0B701C8010E94BE07E4
:10166000882309F44AC080916B01F80127813085F5
:1016700084FF02C0306802C03F77F80130872783BB
:1016800080916B0190E08F709070F8012781308518
:10169000207F26C0B701C8010E94BE07882369F1D8
:1016A00080916B0190E08F709070B4E0880F991F6B
:1016B000BA95E1F7F801278130852F7011C0B70185
:1016C000C8010E94BE078823C1F080916B0190E0A1
:1016D0008F709070982F8827F80127813085307F90
:1016E000822B932B90878783C8010E949B0505C09E
:1016F00067E671E08D2D0E94880840988091640112
:1017000090E09F938F9386E790E09F938F930E9442
:10171000761180916701FFE0DF2ED8222D2D30E079
:1017200082958F7090E03F932F939F938F938EE6D7
:1017300090E09F938F930E94761100E010E08DB7A8
:101740009EB70A960FB6F8949EBF0FBE8DBFE8E60F
:10175000EE2EE0E0FE2E0FC0F0E0E959FE4F808152
:1017600090E09F938F93FF92EF920E9476110F90DB
:101770000F900F900F90E02FEF5F0F5F1F4FD0166D
:1017800058F76091B1037091B2038AE090E00E9433
:101790004A110E941C0F882349F160E08091640186
:1017A0000E94F30CFC01892B09F181858830F1F44A
:1017B000CF010E949B051AC04423C1F0109164011F
:1017C000812F806620E830E03F932F9391E69F932E
:1017D0008F930E9445080F900F900F900F900E94DA
:1017E000FC028823E1F7812F0E94C2021092790146
:1017F0001092780111E060E0812F0E94F30CFC014F
:10180000892B61F08285882349F0893029F48CE0A6
:1018100011928A95E9F702C0818712861F5F103204
:1018200051F70E94FC02882309F08EC09091E601D6
:101830008091E701981721F14091E70182E1489FEB
:101840008001112406581E4FA8014D5F5F4FF8011B
:10185000628180810E945E07F801818181508183CD
:10186000882309F06EC08091E7018F5F8093E701C4
:101870008091E701863008F464C01092E70161C0EE
:1018800080916601882371F4809165018F5F809358
:101890006501803238F0109264011092650181E098
:1018A0008093660180916501882399F06091B1036E
:1018B0007091B2038BE290E00E944A118091650121
:1018C0008093640160E00E94F30C20916501822FF7
:1018D00035C0809164010E943E0D8C010097E9F0B3
:1018E000FC01908180916401891768F08091660104
:1018F0008F5F809366016091B1037091B2038AE0BB
:1019000090E00E944A11F8018081809364018185F2
:10191000863019F4C8010E9486076091B103709166
:10192000B2038EE290E00E944A11809166018F5FBF
:101930008093660180916401882319F080640E947D
:10194000C20284E08093AD0326960FB6F894DEBF02
:101950000FBECDBFDF91CF911F910F91FF90EF9000
:10196000DF900895E0EFF1E0482F50E020E030E014
:101970008081882311F421E030E02417350719F421
:1019800080E090E008953C9682E0E03BF80771F734
:1019900081E090E008958091B0029091B1020895A5
:1019A0009C01E0EFF1E08285882309F4818588308D
:1019B00051F4818192818217930761F08381948130
:1019C0008217930739F03C9682E0E03BF80759F71D
:1019D000E0E0F0E0CF01089580ECE0EFF1E011925B
:1019E0008A95E9F70895CF93DF93482F81508F317F
:1019F00098F5C0EFD1E08881841781F12C9682E0C0
:101A0000C03BD807C1F7662339F1C0EFD1E020E031
:101A100030E088818823D1F4488382E08987822F4F
:101A200090E09F938F93842F90E09F938F938EE706
:101A300090E09F938F930E9476118DB79EB7069684
:101A40000FB6F8949EBF0FBE8DBF08C02C962F5FB7
:101A50003F4F20313105E9F6C0E0D0E0CE01DF9103
:101A6000CF910895882319F480E090E002C00E948D
:101A7000F30C9093B1028093B00208950F931F93DB
:101A8000182F882311F401E005C0803210F00FE117
:101A900001C0082F1F5F103208F011E060E0812FB5
:101AA0000E94F30C101711F00097A1F31F910F91F2
:101AB000089580E090E008958FEF9FEF08950895D6
:101AC00080E090E0089580E090E008958FEF9FEF30
:101AD0000895FC0130E090E08191982720E0892F63
:101AE000869590FF03C097E0982701C0982F2F5F3D
:101AF0002830A9F73F5F383079F797FD9095892F07
:101B000090E008950F931F938C010E94690D20E0CF
:101B1000F8019085891321E081E02827822F90E049
:101B20001F910F910895FC01862F8F778283CA0140
:101B3000892F9927869586958F7366956074862B75
:101B40008383CA0123E0969587952A95E1F78F77DD
:101B500084834295407745830895FC01862F8F77D3
:101B60008083660F672F661F770B71956F77618390
:101B700008950F931F93CF93DF93082F162FEA0139
:101B800002C00E947600AE01612F802F0E94CF0F0D
:101B90008823B9F3DF91CF911F910F910895CF93CF
:101BA000DF93CDB7DEB726970FB6F894DEBF0FBE32
:101BB000CDBFFE01319696E0DF011D929A95E9F7BF
:101BC0004983AF010E94B90D26960FB6F894DEBF87
:101BD0000FBECDBFDF91CF9108959B01AC018091E5
:101BE000A5039091A603A091A703B091A803821723
:101BF0009307A407B507B8F08091A5039091A603B9
:101C0000A091A703B091A80360E070E0821B930B42
:101C1000A40BB50B80509041A040B04010F461E09F
:101C200070E0CB0108958091A5039091A603A09147
:101C3000A703B091A80360E070E0281B390B4A0BA2
:101C40005B0B2050304F4F4F5F4F10F061E070E062
:101C5000CB010895E82FF0E0EF70F070EB56FF4FE6
:101C6000E4918E2F90E00895682F87FF7AC08091CD
:101C7000990390919A03892BE1F0809195038F5FEE
:101C80008093950380919503803110F01092950315
:101C90009091950380919603981759F4809196033B
:101CA0008F5F8093960380919603803110F010929D
:101CB000960380919703909198038B5B924061F01B
:101CC00058F0809194038F5F8093940380919403E4
:101CD000883010F01092940310929A031092990396
:101CE000109298031092970380911201681721F4C3
:101CF00081E080939F0367C010929F03262F30E0FE
:101D00002F773070482F50E02417350729F06F3FA8
:101D100019F08F3F09F057C08091950379E0879FB4
:101D2000C00111248D5F9C4F90939A038093990377
:101D30002417350709F047C09091930380919403CD
:101D4000981741F080919403879FC0011124855416
:101D50009D4F02C082EB92E090939803809397038B
:101D600032C020919F03213029F0213060F12630CC
:101D700050F515C082E080939F03603419F41092EF
:101D8000A00321C0613419F42093A0031CC0623465
:101D900019F0633491F483E08093A00314C0E22F20
:101DA000F0E08091A00390E002968E179F0744F028
:101DB000E756FC4F8081681719F010929F0303C00B
:101DC0002F5F20939F0380919F03882339F4E09134
:101DD0009703F0919803309721F40AC0862F90E082
:101DE00009C0819190E0F0939803E093970302C0BB
:101DF0008FEF9FEF909311018093100180919903D1
:101E000090919A038359934020F010929A03109274
:101E10009903E0919903F0919A03309729F0619327
:101E2000F0939A03E0939903089510929F03109200
:101E300098031092970308959091930380919403CF
:101E400020E030E0981711F421E030E0C901089556
:101E5000DC01209193038091940330E090E001979E
:101E60002817390721F180919303873021F480915D
:101E700094038823E1F09091930389E0989FF00107
:101E80001124E554FD4F90E08D9181939F5F99302F
:101E9000D9F7809193038F5F80939303809193038D
:101EA000883010F01092930381E090E0089580E074
:101EB00090E00895FC01209197033091980390E001
:101EC000A2EBB2E02A173B0720F082E0233B380761
:101ED000C8F380818C939F5F993018F411963196E6
:101EE000F1CF08959C0190919503809196039817E6
:101EF00019F420E030E01FC021153105E1F0F8941D
:101F00009091960389E0989FF0011124ED5FFC4FBA
:101F1000D90190E081918D939F5F9930D9F780919D
:101F200096038F5F8093960380919603803110F023
:101F3000109296037894C90108950E948A019B012A
:101F4000AC0193E0E92FF0E0E556FC4F822F8F774C
:101F5000808387E056954795379527958A95D1F7E1
:101F6000915080F70E944C0308958091A303882329
:101F700019F480E090E008951092A30381E090E0CE
:101F800008952091A1033091A2039093A20380931E
:101F9000A103C90108958091120190E008950F9363
:101FA0001F93CF93DF93CDB7DEB729970FB6F89481
:101FB000DEBF0FBECDBFDA01A89580911201806807
:101FC00089836A83FE0133969E01275F3F4F1097F6
:101FD00021F08D918F77808301C010823196E217B6
:101FE000F307A9F7CE0101960E94690D89878E013A
:101FF0000F5F1F4FC8010E94280F8823D9F381E08B
:1020000090E029960FB6F894DEBF0FBECDBFDF91EA
:10201000CF911F910F9108952F923F924F925F920F
:102020006F927F928F929F92AF92BF92CF92DF92E8
:10203000EF92FF920F931F93CF93DF93CDB7DEB74D
:1020400029970FB6F894DEBF0FBECDBF0E948A015C
:10205000FFE72F2E312C412C512C262237224822EB
:102060005922E0E86E2EEFE37E2E812C912C662221
:1020700077228822992257E09594879477946794E1
:102080005A95D1F7A12C40ECB42E4FE1C42ED12C9F
:10209000A622B722C822D9223EE0D594C794B7948D
:1020A000A7943A95D1F7E12CF12C20EE022F112DB7
:1020B000E622F7220823192385E115950795F79461
:1020C000E7948A95D1F735C0A8958A81843089F53F
:1020D000CE0101960E94820D882359F18E8190E0F5
:1020E000A0E0B0E0281639064A065B0611F58D819E
:1020F00090E0A0E0B0E0681679068A069B06C9F475
:102100008C8190E0A0E0B0E0A816B906CA06DB0614
:1021100081F48B8190E0A0E0B0E0E816F9060A07B0
:102120001B0739F489818F778093120181E090E059
:1021300008C0CE0101960E94720F892B29F680E01B
:1021400090E029960FB6F894DEBF0FBECDBFDF91A9
:10215000CF911F910F91FF90EF90DF90CF90BF90A4
:10216000AF909F908F907F906F905F904F903F9037
:102170002F9008950F931F93CF93DF93CDB7DEB7C2
:1021800029970FB6F894DEBF0FBECDBF8091120124
:102190008F3F11F50E940C10882331F180911201BC
:1021A0000E94AC0321C0C8010E94820D8823B9F0AF
:1021B0008A81863021F481E08093A30310C0E091EE
:1021C000A103F091A203309719F0C801099507C047
:1021D000C8010E94B50303C08E010F5F1F4FC801E5
:1021E0000E94720F892BF9F629960FB6F894DEBF7C
:1021F0000FBECDBFDF91CF911F910F9108950F9327
:102200001F93CF93DF93CDB7DEB729970FB6F8941E
:10221000DEBF0FBECDBF209112012068298323E0CD
:102220002A83282F2F772B83880F892F881F990BBC
:1022300091958F778C83862F8F778D83CA01892F15
:102240009927869586958F738E8367FF02C0806479
:102250008E83CA01A3E096958795AA95E1F78F77BB
:102260008F83842F8295807788878E010F5F1F4F21
:10227000C8010E94690D8987C8010E945A0F2996DA
:102280000FB6F894DEBF0FBECDBFDF91CF911F9187
:102290000F9108950F931F93CF93DF938C01EB0160
:1022A0008B8181FF1BC082FF0DC02E813F818C81FD
:1022B0009D812817390764F4E881F9810193F98336
:1022C000E88306C0E885F985802F0995892B31F4CC
:1022D0008E819F8101969F838E8302C00FEF1FEF37
:1022E000C801DF91CF911F910F910895A2E0B0E056
:1022F000ECE7F1E10C943114FE0137966191719194
:10230000FA83E983E091B103F091B203838188609D
:10231000838349815A818091B1039091B2030E94D5
:102320009C11E091B103F091B2032381277F2383B5
:10233000E2E022960C944D142F923F925F926F929E
:102340007F928F929F92AF92BF92CF92DF92EF9245
:10235000FF920F931F93CF93DF93CDB7DEB72B97E9
:102360000FB6F894DEBF0FBECDBF3C014B016A0132
:10237000FC0117821682838181FD03C08FEF9FEFDE
:10238000BBC11E010894211C311CF3013381F401EF
:1023900033FD859133FF81914F01882309F4A9C151
:1023A000853239F433FD859133FF81914F018532B8
:1023B00029F4B30190E00E944A11E7CF982FAA2494
:1023C00010E055241032B0F49B3269F09C3228F4AE
:1023D000903251F0933271F40BC09D3239F090334A
:1023E00049F411602AC01260146027C0186025C02B
:1023F000106123C017FD2AC0292F20532A3088F4EA
:1024000016FF07C08AE0A89EC0011124A22EA80EC4
:1024100014C08AE0589EC0011124522E580E10623A
:102420000CC09E3221F416FD64C1106406C09C36B7
:1024300011F4106802C0983649F4F40133FD959107
:1024400033FF91914F01992309F0BCCF892F855417
:10245000833018F08052833038F424E030E0C20E2C
:10246000D31E8FE389830FC0933631F0933781F009
:10247000933509F056C020C0F6018081898322E09F
:1024800030E0C20ED31E710181E0A82EB12C12C023
:10249000F601E080F18016FD03C06FEF7FEF02C010
:1024A0006A2D70E022E030E0C20ED31EC7010E9408
:1024B0009F135C011F7713C0F601E080F18016FDC9
:1024C00003C06FEF7FEF02C06A2D70E022E030E0C2
:1024D000C20ED31EC7010E9494135C01106813FF43
:1024E00007C01BC0B30180E290E00E944A115A94D9
:1024F000852D90E0A816B906A8F30FC0F70117FDC7
:10250000859117FF81917F01B30190E00E944A11EC
:1025100051105A940894A108B108A114B10471F79C
:10252000E5C0943611F0993669F517FF0AC0F60137
:10253000608171818281938124E030E0C20ED31EDC
:102540000DC0F601808191819C01B901882777FD3A
:102550008095982F42E050E0C40ED51E012F0F76D3
:1025600097FF08C090958095709561957F4F8F4F2C
:102570009F4F00682AE030E0A1010E94AA13B82E04
:10258000B2183DC0953721F41F7E2AE030E01CC010
:10259000197F9F3661F0903720F4983509F0A9C073
:1025A0000FC0903739F0983709F0A3C004C028E075
:1025B00030E00AC0106114FD146020E130E004C076
:1025C00014FD166020E132E017FF08C0F6016081BB
:1025D00071818281938144E050E008C0F6018081DE
:1025E0009181BC0180E090E042E050E0C40ED51E35
:1025F000A1010E94AA13B82EB218012F0F7706FF6F
:1026000009C00E7FBA1430F404FF06C002FD04C0F6
:102610000F7E02C01B2D01C01A2D04FF0CC0FE014D
:10262000EB0DF11D8081803311F4097E08C01F5F1E
:1026300002FF05C003C0802F867809F01F5FE02EDF
:1026400003FD14C000FF0FC0151510F0AB2C0BC01C
:10265000AB2CA50CA11A152D06C0B30180E290E0A9
:102660000E944A111F5F1515C0F304C0151510F420
:10267000511A01C05524E4FE10C0B30180E390E07C
:102680000E944A11E2FE1EC0E1FE03C088E590E010
:1026900002C088E790E0B3010CC08E2D867891F0DF
:1026A000E1FE02C08BE201C080E207FD8DE2B301D2
:1026B00090E00E944A1106C0B30180E390E00E94BE
:1026C0004A11AA94BA14C0F3BA94F101EB0DF11DAA
:1026D0008081B30190E00E944A11BB2039F0F4CF11
:1026E000B30180E290E00E944A115A945520C1F74C
:1026F0004CCEF301868197812B960FB6F894DEBFFE
:102700000FBECDBFDF91CF911F910F91FF90EF9042
:10271000DF90CF90BF90AF909F908F907F906F9001
:102720005F903F902F900895FC010590615070409C
:102730000110D8F7809590958E0F9F1F0895FC018A
:102740006150704001900110D8F7809590958E0FE0
:102750009F1F0895FA01AA27283051F1203181F1F5
:10276000E8946F936E7F6E5F7F4F8F4F9F4FAF4F99
:10277000B1E03ED0B4E03CD0670F781F891F9A1FAC
:10278000A11D680F791F8A1F911DA11D6A0F711D60
:10279000811D911DA11D20D009F468943F912AE06C
:1027A000269F11243019305D3193DEF6CF01089554
:1027B000462F4770405D4193B3E00FD0C9F7F6CF85
:1027C000462F4F70405D4A3318F0495D31FD40524D
:1027D000419302D0A9F7EACFB4E0A69597958795E3
:1027E00077956795BA95C9F70097610571050895C2
:1027F0009B01AC010A2E069457954795379527956E
:10280000BA95C9F7620F731F841F951FA01D089505
:10281000F999FECFB2BDA1BDF89A119600B4089502
:10282000F7DF01921A94E1F70895F999FECFB2BD4E
:10283000A1BD00BC11960FB6F894FA9AF99A0FBE92
:1028400008952F923F924F925F926F927F928F9254
:102850009F92AF92BF92CF92DF92EF92FF920F932F
:102860001F93CF93DF93CDB7DEB7CA1BDB0B0FB639
:10287000F894DEBF0FBECDBF09942A8839884888F6
:102880005F846E847D848C849B84AA84B984C8848C
:10289000DF80EE80FD800C811B81AA81B981CE0F83
:1028A000D11D0FB6F894DEBF0FBECDBFED01089568
:0228B000FFCF58
:1028B2000080800080000080800000800080800016
:0428C200FFFFFF0015
:00000001FF
